:020000040000FA
:040000008EEF00F08F
:100008004382FACF15F0FBCF16F0E1CF17F0E2CF1D
:1000180018F0D9CF19F0DACF1AF0F3CF1BF0F4CFDC
:100028001CF0F2AA1AEF00F01CEF00F027EF00F026
:10003800F2A421EF00F023EF00F027EF00F0CAEC64
:1000480017F07CEF00F0F2AC2CEF00F02EEF00F090
:100058007CEF00F09DA233EF00F035EF00F040EFA9
:1000680000F09EA23AEF00F03CEF00F040EF00F005
:1000780048EC18F07CEF00F09DAA45EF00F047EF40
:1000880000F05EEF00F09EAA4CEF00F04EEF00F09B
:100098005EEF00F002D85CEF00F005000001FA6E98
:1000A800AC51FD6EAD51FE6EF850FF6EFA50120065
:1000B8007CEF00F09DA863EF00F065EF00F07CEFA7
:1000C80000F09EA86AEF00F06CEF00F07CEF00F003
:1000D80002D87AEF00F005000001FA6EAA51FD6E11
:1000E800AB51FE6EF850FF6EFA5012007CEF00F034
:1000F8001CC0F4FF1BC0F3FF1AC0DAFF19C0D9FFF8
:1001080018C0E2FF17C0E1FF16C0FBFF15C0FAFFD9
:1001180043921100A3EF07F00001646F61EC1AF03D
:100128000009D8B49AEF00F09CEF00F09FEF00F0C0
:10013800100E36EC1CF0000164514AEC1CF08EEFF6
:1001480001F000016405D8B4ACEF00F0AEEF00F0A8
:10015800B3EF00F0110E5DEC1BF0B7EF01F098EC77
:100168001CF0010E316EB7EF01F0300E000164197A
:10017800D8B4C1EF00F0C3EF00F0C8EF00F0120EE2
:100188005DEC1BF0B7EF01F0020E316EB7EF01F036
:10019800610E1D6E000E1E6E00016451FCEC13F022
:1001A8000001636F6351D8B4DCEF00F0DEEF00F0BC
:1001B800E3EF00F063515DEC1BF0B7EF01F064C0B2
:1001C800B2F020EE02F06151D9266251DA22DF50F6
:1001D800306E3050D8B4F3EF00F0F5EF00F0FBEFDD
:1001E80000F0030E316E000E2F6EB7EF01F0050E12
:1001F800316EB7EF01F0400E206E000E216E000147
:1002080064517DEC10F00001636F6351D8B40FEFB7
:1002180001F011EF01F016EF01F063515DEC1BF0F6
:10022800B7EF01F0040E316EB7EF01F03F0E206E0C
:10023800000E216E000164517DEC10F00001636F27
:100248006351D8B42AEF01F02CEF01F031EF01F03F
:1002580063515DEC1BF0B7EF01F04050100DF35007
:100268003F24606FEF0E2F643CEF01F03EEF01F08A
:1002780043EF01F0140E5DEC1BF0B7EF01F0000E38
:100288002F24D96EDA6A030EDA2260C0DFFF2F2A24
:1002980030063050D8A453EF01F055EF01F057EF76
:1002A80001F0FBEF00F0030E316EB7EF01F0C3EC85
:1002B8001CF00009D8B463EF01F065EF01F06AEFB4
:1002C80001F0150E5DEC1BF0B7EF01F00001645171
:1002D800D8A471EF01F073EF01F077EF01F0070E8A
:1002E800316EB7EF01F0060E316EB7EF01F0000185
:1002F8006451D8B482EF01F084EF01F073EF01F09C
:10030800160E5DEC1BF0B7EF01F0170E5DEC1BF05D
:10031800B7EF01F03150246E256A2550000AD8B491
:1003280098EF01F089EF01F02450000AD8B4A5EF46
:1003380000F0010AD8B4B9EF00F0030AD8B4CCEF42
:1003480000F0010AD8B4FFEF00F0070AD8B41AEF9A
:1003580001F0010AD8B45BEF01F0030AD8B47BEFCF
:1003680001F089EF01F0120020EE02F00350D926C7
:100378000450DA2203C0E1FF04C0E2FF02D8CFEF45
:1003880001F00500FA6EE650FD6EE650FE6EF8507C
:10039800FF6EFA501200DF6E20EE02F00350D926ED
:1003A8000450DA2210EE03F00350E1260450E22252
:1003B800DE50E65CD8B0E3EF01F0E5EF01F0F3EFD3
:1003C80001F020EE02F00350D9260450DA2210EE94
:1003D80003F00350E1260450E222DFCFE7FF20EECE
:1003E80004F00350D9260450DA22DF50D8B4FFEFC6
:1003F80001F001EF02F0C6EF02F020EE02F0035028
:10040800D9260450DA22DF50D8B40DEF02F00FEFEE
:1004180002F059EF02F020EE08F00350D9260450FC
:10042800DA22DE2A000EDD2220EE08F00350D9265B
:100438000450DA22DE50DE10D8A425EF02F027EFB0
:1004480002F030EF02F020EE08F00350D9260450F5
:10045800DA22DE06000EDD5A20EE08F00350D92617
:100468000450DA2210EE0AF00350E1260450E2228A
:10047800DE50E65CDE50E658D8B045EF02F047EFB4
:1004880002F063EF02F020EE08F00350D926045082
:10049800DA2210EE0AF00350E1260450E222DECF01
:1004A800E6FFDDCFE5FF63EF02F020EE08F0035032
:1004B800D9260450DA22000EDE6E000EDD6E20EE24
:1004C80005F00350D9260450DA22DF50D8B46FEF74
:1004D80002F071EF02F0C6EF02F020EE08F00350D0
:1004E800D9260450DA2210EE06F00350E126045013
:1004F800E222DE50E65CDE50E658D8B086EF02F025
:1005080088EF02F0C6EF02F020EE0CF00350D92677
:100518000450DA2202D89BEF02F00500FA6EDE5092
:10052800FD6EDE50FE6EF850FF6EFA50120020EE9F
:100538000EF00350D9260450DA22DE2A000EDD22FE
:1005480020EE0EF00350D9260450DA22DE50DE10D9
:10055800D8A4B1EF02F0B3EF02F0BCEF02F020EE46
:100568000EF00350D9260450DA22DE06000EDD5ABA
:1005780020EE08F00350D9260450DA22000EDE6E71
:10058800000EDD6E120000000000000000000000F8
:100598000000000000000000000000000000000053
:1005A8000000000000000000000000000000005AE9
:1005B80039010000000000000000000000000000F9
:1005C8000000000000000000000000000000000023
:1005D800000000000000000000005A39020000007E
:1005E8000000000000000000000000000000000003
:1005F80000000000000000000000000000000000F3
:1006080000000000005A390300000000000000004C
:100618000000000000000000010110F902000000C5
:1006280000000000010170B7090000000000000090
:10063800083804000000000000000000000000006E
:10064800000000010180F20200000000000000012B
:1006580001E0B00900000000000000FE37050000BE
:100668000000000000000000000000000000010081
:1006780018F60300000000000000010078691C0063
:100688000000000000004E390600000000000000D5
:100698000000000000000000000000000000000052
:1006A8000000000000000000000000000000000042
:1006B800005A390700000000000000000000000098
:1006C80000000000010012F103000000000000001B
:1006D8000100E5C81C0000000000000048390800BF
:1006E8000000000000000000000000000000000002
:1006F80000000000000000000000000000000000F2
:10070800000000000000005A390900000000000045
:1007180000000000000000000000000000000000D1
:1007280000000000000000000000000000000000C1
:1007380000005A390A000000000000000000000014
:1007480000000000000000000000000000000000A1
:0F075800000000000000000000000000005A39FF
:100768008FEC1AF000016D6F6D51D8A4BEEF03F045
:10077800C0EF03F0C3EF03F0020E6BEF04F0170EA7
:100788006D65C9EF03F0CBEF03F0CDEF03F0C0EFD9
:1007980003F06DC060F06D519EEC11F00009D8B403
:1007A800D8EF03F0DAEF03F023EF04F000016D5106
:1007B80020EC07F01FC06BF020C06CF0F29E000127
:1007C80020EE01F06B51D9266C51DA22DECF61F0B0
:1007D800DDCF62F020EE0DF06B51D9266C51DA2294
:1007E800DECF63F0DDCF64F020EE0FF06B51D92639
:1007F8006C51DA22DECF65F0DDCF66F020EE07F02F
:100808006B51D9266C51DA22DECF24F0DECF25F0E9
:10081800DECF26F0DECF27F04250E82A19EF04F0A9
:10082800D8902732263225322432E82E14EF04F0ED
:1008380024C067F025C068F0F28E4CEF04F0000188
:100848006D518AEC05F01FC069F020C06AF0F29E75
:10085800000120EE02F06951D9266A51DA22DF50F0
:10086800246E2450616F626B000E646F000E636F1C
:1008780020EE03F06951D9266A51DA22DF50246E3E
:100888002450656F666B000E686F000E676FF28EFE
:1008980095EC1CF00001605184EC1AF061C01DF069
:1008A80062C01EF004EC19F063C01DF064C01EF0B5
:1008B80004EC19F065C01DF066C01EF004EC19F0D8
:1008C80067C01DF068C01EF004EC19F0000E12009D
:1008D800000E0001866F000E876F010E8A6F8A5125
:1008E8009EEC11F00009D8B47CEF04F07EEF04F020
:1008F8009EEF04F000018A5120EC07F01FC082F03F
:1009080020C083F0F29E000120EE01F08251D9262A
:100918008351DA228651020D6C0EF324E16E000E2B
:10092800F420E26EDECFE6FFDDCFE5FFF28E862B08
:10093800B8EF04F000018A518AEC05F01FC084F07A
:1009480020C085F0F29E000120EE02F08451D926E5
:100958008551DA22600E8725E16EE26A000EE222F6
:10096800DFCFE7FFF28E872B8A2B170E8A65BFEF42
:1009780004F0C1EF04F073EF04F095EC1CF0000EE6
:100988000001886FD8EF04F08851020D6C0EF32433
:10099800D96E000EF420DA6EDECF1DF0DDCF1EF02A
:1009A80004EC19F00001882B8651885DD8A0DFEF90
:1009B80004F0E1EF04F0C8EF04F0000E896FF0EFE7
:1009C80004F0600E8925D96EDA6A000EDA22DF504B
:1009D80084EC1AF00001892B8751895DD8A0F7EFC4
:1009E80004F0F9EF04F0E5EF04F0000E1200000E39
:1009F8000001866F000E876F010E8A6F8A519EEC88
:100A080011F00009D8B40BEF05F00DEF05F02DEF4C
:100A180005F000018A5120EC07F01FC082F020C0C9
:100A280083F0F29E000120EE0FF08251D926835107
:100A3800DA228651020D6C0EF324E16E000EF420CA
:100A4800E26EDECFE6FFDDCFE5FFF28E862B47EFC5
:100A580005F000018A518AEC05F01FC084F020C01F
:100A680085F0F29E000120EE03F08451D9268551CD
:100A7800DA22600E8725E16EE26A000EE222DFCFFD
:100A8800E7FFF28E872B8A2B170E8A654EEF05F04B
:100A980050EF05F002EF05F095EC1CF0000E000198
:100AA800886F67EF05F08851020D6C0EF324D96E3C
:100AB800000EF420DA6EDECF1DF0DDCF1EF004EC60
:100AC80019F00001882B8651885DD8A06EEF05F0DB
:100AD80070EF05F057EF05F0000E896F7FEF05F016
:100AE800600E8925D96EDA6A000EDA22DF5084ECAE
:100AF8001AF00001892B8751895DD8A086EF05F08F
:100B080088EF05F074EF05F0000E1200236ED9EFA0
:100B180005F0000E1F6E010E206E16EF06F0100E87
:100B28001F6E010E206E16EF06F0200E1F6E010ECE
:100B3800206E16EF06F0300E1F6E010E206E16EFB7
:100B480006F0400E1F6E010E206E16EF06F0500ED6
:100B58001F6E010E206E16EF06F0600E1F6E010E5E
:100B6800206E16EF06F0700E1F6E010E206E16EF47
:100B780006F0800E1F6E010E206E16EF06F0900E26
:100B88001F6E010E206E16EF06F0A00E1F6E010EEE
:100B9800206E16EF06F0B00E1F6E010E206E16EFD7
:100BA80006F07FEC16F08DEF05F02350216E226AD7
:100BB8002250000AD8B4E3EF05F0D5EF05F0215034
:100BC8000C0AD8B48DEF05F0010AD8B493EF05F0FC
:100BD800030AD8B499EF05F0010AD8B49FEF05F0DD
:100BE8001F0AD8B4A5EF05F0010AD8B4ABEF05F099
:100BF800030AD8B4B1EF05F0010AD8B4B7EF05F08D
:100C0800070AD8B4BDEF05F0010AD8B4C3EF05F060
:100C1800030AD8B4C9EF05F0010AD8B4CFEF05F03C
:100C2800D5EF05F0120034502B0DBE0EF3240F6ED5
:100C3800040EF420106E20EE01F00F50D92610504B
:100C4800DA2210EE0FF00F50E1261050E222DE50AB
:100C5800E65CDE50E658D8B034EF06F036EF06F022
:100C680046EF06F020EE01F00F50D9261050DA2298
:100C780010EE0FF00F50E1261050E222DECFE6FF13
:100C8800DDCFE5FF110E0F24016E000E1020026E5D
:100C980020EE01F00F50D9261050DA22DECF03F0F3
:100CA800DDCF04F017EC0BF01D0E0F24016E000EC3
:100CB8001020026E20EE01F00F50D9261050DA22D3
:100CC800DECF03F0DDCF04F017EC0BF0110E0F248C
:100CD800036E000E1020046E20EE29F00F50D92666
:100CE8001050DA22DECF05F0DDCF06F0AAEC0CF0CA
:100CF8000009D8A482EF06F084EF06F096EF06F01C
:100D08001D0E0F24036E000E1020046E20EE29F035
:100D18000F50D9261050DA22DECF05F0DDCF06F0CD
:100D2800AAEC0CF00FC001F010C002F0CBEC0DF0F3
:100D380012008FEC1AF00001676F8FEC1AF00001B7
:100D4800646F6751D8A4ABEF06F0ADEF06F0B0EFD3
:100D580006F0020E1FEF07F00E0E6765B6EF06F0FD
:100D6800B8EF06F0BAEF06F0ADEF06F0020E6465D4
:100D7800C0EF06F0C2EF06F0C4EF06F0ADEF06F0E4
:100D880067C062F067514DEC17F024C065F025C0CC
:100D980066F0F29EF9EF06F065C0D9FF66C0DAFF8B
:100DA800000EDF6E000E636F13EF07F065C0D9FF0A
:100DB80066C0DAFF010EDF6E010E636F13EF07F0F6
:100DC80065C0D9FF66C0DAFFDE04D8B4EEEF06F0DE
:100DD800F1EF06F0010EF2EF06F0000E636F13EF6D
:100DE80007F0F28E010E1FEF07F000016451606FEB
:100DF800616B6151000AD8B404EF07F0F5EF06F013
:100E08006051000AD8B4D0EF06F0010AD8B4DAEF7E
:100E180006F0030AD8B4E4EF06F0F5EF06F0F28E18
:100E280095EC1CF00001625184EC1AF0000163514A
:100E380084EC1AF0000E1200236E69EF07F0BE0E64
:100E48001F6E040E206EA2EF07F0E90E1F6E040E4F
:100E5800206EA2EF07F0140E1F6E050E206EA2EF93
:100E680007F03F0E1F6E050E206EA2EF07F06A0E08
:100E78001F6E050E206EA2EF07F0950E1F6E050E71
:100E8800206EA2EF07F0C00E1F6E050E206EA2EFB7
:100E980007F0EB0E1F6E050E206EA2EF07F0160E80
:100EA8001F6E060E206EA2EF07F0410E1F6E060E93
:100EB800206EA2EF07F06C0E1F6E060E206EA2EFDA
:100EC80007F07FEC16F023EF07F02350216E226A1B
:100ED8002250000AD8B473EF07F065EF07F02150ED
:100EE800010AD8B423EF07F0030AD8B429EF07F0B2
:100EF800010AD8B42FEF07F0070AD8B435EF07F086
:100F0800010AD8B43BEF07F0030AD8B441EF07F061
:100F1800010AD8B447EF07F00F0AD8B44DEF07F02D
:100F2800010AD8B453EF07F0030AD8B459EF07F011
:100F3800010AD8B45FEF07F065EF07F012008E0ED4
:100F4800F66E050EF76E000EF86E04EEBEF011EEAA
:100F5800D9F00900F5CFEEFFE550E150FAE1E25093
:100F6800F8E1D80EF66E1A0EF76E000EF86E04EE63
:100F780000F010EEBEF00900F5CFEEFFE550E150AD
:100F8800FAE1180EF66E1A0EF76E000EF86E01EE04
:100F980000F010EEC0F00900F5CFEEFFE550E1508B
:100FA800FAE1AC0EF66E360EF76E000EF86E00EE35
:100FB800B3F010EE0EF00900F5CFEEFFE550E1506A
:100FC800FAE1960EF66E390EF76E000EF86E09000D
:100FD800F5CF41F00900F5CF42F003EE00F0F00E36
:100FE800EE6AE806FDE102EE00F0800EEE6AE80621
:100FF800FDE101EEC0F0400EEE6AE806FDE100EE0C
:1010080090F0230EEE6AE806FDE100EE28F0190ED6
:10101800EE6AE806FDE143904392000EF86E000187
:1010280060EF18F08FEC1AF00001696F6951D8A4CD
:1010380020EF08F022EF08F025EF08F0020E87EF06
:1010480008F00F0E69652BEF08F02DEF08F02FEF71
:1010580008F022EF08F069C066F0000E676F0F0E07
:101068006919D8A43AEF08F03CEF08F063EF08F0EC
:10107800010E686F68512CEC17F024C062F025C08F
:1010880063F0F29E62C0D9FF63C0DAFFDE50DE1063
:10109800D8B451EF08F053EF08F056EF08F0010EFE
:1010A8000001676FF28E0001682B0E0E68655FEF16
:1010B80008F061EF08F03EEF08F07CEF08F06951A6
:1010C8002CEC17F024C064F025C065F0F29E64C0D3
:1010D800D9FF65C0DAFFDE50DE10D8B476EF08F02D
:1010E80078EF08F07BEF08F0010E0001676FF28ED1
:1010F80095EC1CF00001665184EC1AF00001675170
:1011080084EC1AF0000E12003550D8A48EEF08F0C7
:1011180090EF08F092EF08F0F8EF08F0330633503C
:10112800D8B499EF08F09BEF08F0E3EF08F0F8EF78
:1011380008F032EC1BF00009D8A4A5EF08F0A7EFDF
:1011480008F0AAEF08F0332AF8EF08F03CEC1BF09F
:1011580001C013F002C014F034502B0DBF0EF3245D
:10116800D96E040EF420DA6E13C0DEFF14C0DDFF62
:1011780017EC06F0010E3424016E026A000E0222FA
:10118800000E046E0B0E036E80EC0EF00150346EF0
:1011980034502B0DBE0EF324D96E040EF420DA6EF3
:1011A800DF506DEC1AF0020E356E010E336EF8EF5B
:1011B80008F0C9EC1CF0010E356ED9EF08F0355077
:1011C800116E126A1250000AD8B4EDEF08F0F8EF69
:1011D80008F01150010AD8B49DEF08F0030AD8B4FA
:1011E800DDEF08F0F8EF08F012008FEC1AF00001BC
:1011F800676F8FEC1AF00001666F6751D8A407EF8C
:1012080009F009EF09F00CEF09F0020E68EF09F098
:10121800080E676512EF09F014EF09F016EF09F0F0
:1012280009EF09F0020E66651CEF09F01EEF09F0E0
:1012380020EF09F009EF09F067C064F067517DEC11
:101248000BF01FC060F020C061F000016751E2ECB4
:101258000BF01FC062F020C063F0020E0001661997
:10126800D8B439EF09F03BEF09F04BEF09F0F29EE3
:1012780002D84AEF09F00500FA6E6051FD6E61511F
:10128800FE6EF850FF6EFA5066511200F28EF29E12
:1012980002D85AEF09F005000001FA6E6251FD6E9E
:1012A8006351FE6EF850FF6EFA5012000001656F30
:1012B800F28E95EC1CF00001645184EC1AF00001E8
:1012C800655184EC1AF0000E12008FEC1AF0000140
:1012D800646F6451D8A473EF09F075EF09F078EFE3
:1012E80009F0020ED7EF09F0180E64657EEF09F0D9
:1012F80080EF09F082EF09F075EF09F0010E656FD4
:10130800180E6419D8B48BEF09F08DEF09F096EF39
:1013180009F065516419D8A494EF09F096EF09F023
:10132800CBEF09F065519EEC11F00009D8B49FEF9E
:1013380009F0A1EF09F0B8EF09F00001655120ECC0
:1013480007F01FC060F020C061F0F29E000120EE9F
:101358000FF06051D9266151DA22000EDE6E000EC0
:10136800DD6EF28ECBEF09F0000165518AEC05F0D5
:101378001FC062F020C063F0F29E000120EE03F06F
:101388006251D9266351DA22000EDF6EF28E652B88
:10139800170E6565D2EF09F0D4EF09F084EF09F074
:1013A80095EC1CF0000E12008FEC1AF00001626F31
:1013B8006251D8A4E2EF09F0E4EF09F0E7EF09F091
:1013C800020E42EF0AF00E0E6265EDEF09F0EFEF44
:1013D80009F0F1EF09F0E4EF09F0F29E62C042F083
:1013E80042C024F0010E256E000E266E242A00EF5E
:1013F8000AF0D89025362636242EFDEF09F025C0B0
:10140800BFF026C0C0F0F28E010E0001636F635179
:101418009EEC11F00009D8B414EF0AF016EF0AF0A8
:1014280035EF0AF00001635120EC07F01FC060F0AF
:1014380020C061F0F29E000120EE0BF06051D92629
:101448006151DA22000EDE6E000EDD6E20EE03F032
:101458006051D9266151DA22DE6ADE6ADE6ADD6A07
:10146800F28E0001632B170E63653DEF0AF03FEF24
:101478000AF00BEF0AF095EC1CF0000E1200000EBB
:101488000001786F010E7A6F7A519EEC11F0000915
:10149800D8B451EF0AF053EF0AF085EF0AF00001D3
:1014A8007A5120EC07F01FC076F020C077F0F29E4A
:1014B800000120EE07F07651D9267751DA22DECFE7
:1014C80024F0DECF25F0DECF26F0DECF27F0425025
:1014D800E82A74EF0AF0D8902732263225322432CF
:1014E800E82E6FEF0AF07851020D600EF324D96EE2
:1014F800000EF420DA6E24C0DEFF25C0DDFFF28E78
:10150800782B00017A2B170E7A658DEF0AF08FEF92
:101518000AF048EF0AF0000E796FA3EF0AF079514C
:10152800020D600EF324D96E000EF420DA6EDECFC1
:101538001DF0DDCF1EF004EC19F00001792B785175
:10154800795DD8A0AAEF0AF0ACEF0AF093EF0AF0A1
:10155800000E1200236EE9EF0AF0500E1F6E050E02
:10156800206E16EF0BF05C0E1F6E050E206E16EF48
:101578000BF07B0E1F6E050E206E16EF0BF0870E1C
:101588001F6E050E206E16EF0BF0A60E1F6E050ED1
:10159800206E16EF0BF0B20E1F6E050E206E16EFC2
:1015A8000BF0FC0E1F6E050E206E16EF0BF0080EEA
:1015B8001F6E060E206E16EF0BF07FEC16F0DB0E9A
:1015C8001F6E040E206E16EF0BF02350216E226A58
:1015D8002250000AD8B4F3EF0AF0E1EF0AF02150E4
:1015E800010AD8B4B7EF0AF0030AD8B4B1EF0AF089
:1015F800010AD8B4C3EF0AF0070AD8B4BDEF0AF05D
:10160800010AD8B4CFEF0AF0030AD8B4C9EF0AF038
:10161800010AD8B4DBEF0AF00F0AD8B4D5EF0AF004
:10162800E1EF0AF0120020EE02F00150D926025034
:10163800DA220350DE5C0450DE58D8B026EF0BF0F7
:1016480028EF0BF072EF0BF020EE06F00150D926D0
:101658000250DA22DE2A000EDD2220EE06F00150CA
:10166800D9260250DA22DE50DE10D8A43EEF0BF065
:1016780040EF0BF049EF0BF020EE06F00150D926B1
:101688000250DA22DE06000EDD5A20EE06F0015086
:10169800D9260250DA2210EE08F00150E126025055
:1016A800E222DE50E65CDE50E658D8B05EEF0BF082
:1016B80060EF0BF07CEF0BF020EE06F00150D9261E
:1016C8000250DA2210EE08F00150E1260250E22220
:1016D800DECFE6FFDDCFE5FF7CEF0BF020EE06F076
:1016E8000150D9260250DA22000EDE6E000EDD6EA1
:1016F8001200236EB0EF0BF01E0E1F6E340E206E1C
:10170800E1EF0BF0FE0E1F6E330E206EE1EF0BF0D3
:10171800DE0E1F6E330E206EE1EF0BF0BE0E1F6E55
:10172800330E206EE1EF0BF09E0E1F6E330E206E0F
:10173800E1EF0BF07E0E1F6E330E206EE1EF0BF023
:101748005E0E1F6E330E206EE1EF0BF03E0E1F6E25
:10175800330E206EE1EF0BF02350216E226A2250E7
:10176800000AD8B4BAEF0BF0DDEF0BF02150010AF4
:10177800D8B480EF0BF0030AD8B486EF0BF0010A57
:10178800D8B48CEF0BF0070AD8B492EF0BF0010A2B
:10179800D8B498EF0BF0030AD8B49EEF0BF0010A07
:1017A800D8B4A4EF0BF00F0AD8B4AAEF0BF0DDEF12
:1017B8000BF07FEC16F0AAEF0BF01200236E15EF7A
:1017C8000CF0120E1F6E390E206E46EF0CF00C0E48
:1017D8001F6E390E206E46EF0CF0060E1F6E390E86
:1017E800206E46EF0CF0000E1F6E390E206E46EF8D
:1017F8000CF0FA0E1F6E380E206E46EF0CF0F40E49
:101808001F6E380E206E46EF0CF0EE0E1F6E380E6F
:10181800206E46EF0CF0E80E1F6E380E206E46EF75
:101828000CF02350216E226A2250000AD8B41FEF10
:101838000CF042EF0CF02150010AD8B4E5EF0BF0A0
:10184800030AD8B4EBEF0BF0010AD8B4F1EF0BF0B0
:10185800070AD8B4F7EF0BF0010AD8B4FDEF0BF084
:10186800030AD8B403EF0CF0010AD8B409EF0CF05E
:101878000F0AD8B40FEF0CF042EF0CF07FEC16F023
:101888000FEF0CF01200C00E3924D96EDA6A010E7F
:10189800DA22000EDF6EABA454EF0CF056EF0CF01A
:1018A8006CEF0CF0C00E3924D96EDA6A010EDA2218
:1018B8000101DF8202D86CEF0CF005000001FA6E1E
:1018C800A851FD6EA951FE6EF850FF6EFA50120035
:1018D800ABA271EF0CF073EF0CF089EF0CF0C00EB7
:1018E8003924D96EDA6A010EDA220101DF8402D8BE
:1018F80089EF0CF005000001FA6EA651FD6EA751A4
:10190800FE6EF850FF6EFA501200C00E3924D96EE0
:10191800DA6A010EDA22DF50D8B495EF0CF097EFAF
:101928000CF0A7EF0CF002D8A5EF0CF005000001B1
:10193800FA6EA451FD6EA551FE6EF850FF6EFA5076
:101948001200A9EF0CF0A2EC18F0120020EE01F042
:101958000350D9260450DA22DF50D8B4B6EF0CF081
:10196800B8EF0CF00AEF0DF020EE06F00350D92680
:101978000450DA2210EE04F00350E1260450E2226B
:10198800DE50E65CDE50E658D8B0CDEF0CF0CFEF75
:101998000CF00AEF0DF002D8DCEF0CF00500FA6E3F
:1019A8000550FD6E0650FE6EF850FF6EFA5012009C
:1019B80020EE0AF00350D9260450DA22DE2A000E5F
:1019C800DD2220EE0AF00350D9260450DA22DE5038
:1019D800DE10D8A4F2EF0CF0F4EF0CF0FDEF0CF0F1
:1019E80020EE0AF00350D9260450DA22DE06000E53
:1019F800DD5A20EE06F00350D9260450DA22000EF4
:101A0800DE6E000EDD6E010E0BEF0DF0000E120003
:101A18003C360000010105000000000030380000DD
:101A280028360000010105000000000026380000EB
:101A38001436000001010500000000001C380000F9
:101A48000036000001010500000000001238000007
:101A5800EC350000010108000000000054390000C6
:101A6800D8350000010108000000000060390000BE
:101A7800C435000000000000000000005A390000D2
:101A8800B035000000000000000000005A390000D6
:101A98009C35000000000000000000005A390000DA
:101AA8008835000000000000000000005A390000DE
:101AB8007435000000000000000000005A390000E2
:101AC8005036000000000000000000005A390000F5
:101AD800404102F2114243023A0D44450348294667
:101AE800470110274849019C264A4B010A1F4C4DC3
:101AF800036A284E4F01B2255051012C1052530150
:101B08005E1E54550128265657006E2C5859007EE3
:101B18002B5A5B00762A5C5D00CE2B5E5F0168075E
:101B2800606101D212626300D80864650086146699
:101B380067004C1C686900F6096A6B01B0136C6D8C
:101B480000F2346E6F0060307071003030727300D4
:101B58003A257475007834767701B0227879006E6A
:101B6800317A7B00EE367C7D02BE327E7F00DE322B
:101B7800808102C223828301AA34848504B62C861C
:101B88008720B2298889004224000000000020EE46
:101B980001F00150D9260250DA22DECF03F0DDCF62
:101BA80004F020EE03F00150D9260250DA22035047
:101BB800DE260450DE22000EDE22DE2220EE0BF0AE
:101BC8000150D9260250DA22DE2A000EDD2220EE4C
:101BD8000BF00150D9260250DA220001BF51DE5C19
:101BE800C051DE58D8A0FBEF0DF0FDEF0DF025EF4A
:101BF8000EF020EE03F00150D9260250DA2210EE42
:101C080007F00150E1260250E222DECFE6FFDECFE8
:101C1800E6FFDECFE6FFDECFE6FF20EE03F0015061
:101C2800D9260250DA22DE6ADE6ADE6ADD6A20EE32
:101C38000BF00150D9260250DA22000EDE6E000E9B
:101C4800DD6E1200000E0001786F010E7A6F7A5176
:101C58009EEC11F00009D8B434EF0EF036EF0EF018
:101C680054EF0EF000017A5120EC07F01FC076F017
:101C780020C077F0F29E000120EE0DF07651D926B3
:101C88007751DA227851020D600EF324E16E000ECE
:101C9800F420E26EDECFE6FFDDCFE5FFF28E782B93
:101CA80000017A2B170E7A655CEF0EF05EEF0EF0EE
:101CB8002BEF0EF095EC1CF0000E0001796F75EF1C
:101CC8000EF07951020D600EF324D96E000EF42047
:101CD800DA6EDECF1DF0DDCF1EF004EC19F0000146
:101CE800792B7851795DD8A07CEF0EF07EEF0EF05D
:101CF80065EF0EF0000E1200000E066E02BE89EFB0
:101D08000EF087EF0EF08FEF0EF0016C021ED8B0C8
:101D1800022A010E066E04BE96EF0EF094EF0EF046
:101D28009AEF0EF0036C041ED8B0042A0350041076
:101D3800D8B4A1EF0EF0A3EF0EF0C7EF0EF0010E2E
:101D4800056EABEF0EF0D89003360436052A04AEC4
:101D5800B0EF0EF0B2EF0EF0A7EF0EF00350015CFB
:101D680004500258D8A0BBEF0EF0BDEF0EF0C1EF43
:101D78000EF00350015E0450025AD8900432033228
:101D8800052EB2EF0EF00650D8B4CDEF0EF0CFEF1F
:101D98000EF0D3EF0EF0016C021ED8B0022A01C07B
:101DA80001F002C002F012004150D8B4DEEF0EF08C
:101DB800E0EF0EF02EEF0FF0DEEC18F00001BD5151
:101DC800606FBE51616F626B636B1D50605D1E502A
:101DD80061591F50625920506359D8B0F6EF0EF080
:101DE800F8EF0EF027EF0FF0010E2D6E050E2C60A8
:101DF80000EF0FF002EF0FF02EEF0FF071EC1BF079
:101E08000009D8A40AEF0FF00CEF0FF02EEF0FF037
:101E18002C50020DB30EF324D96E000EF420DA6EA6
:101E280002D821EF0FF00500FA6EDE50FD6EDE508D
:101E3800FE6EF850FF6EFA5012003C0E6BEC1BF071
:101E48002C2A2EEF0FF0000E2C6E000E6BEC1BF000
:101E58002EEF0FF012008FEC1AF00001656F65513C
:101E6800D8A439EF0FF03BEF0FF03EEF0FF0020E62
:101E780084EF0FF00F0E656544EF0FF046EF0FF09B
:101E880048EF0FF03BEF0FF00F0E6519D8A44FEF96
:101E98000FF051EF0FF070EF0FF0010E646F645107
:101EA8002CEC17F024C060F025C061F0F29E60C0F1
:101EB800D9FF61C0DAFF000EDE6E000EDD6EF28E15
:101EC8000001642B0E0E64656CEF0FF06EEF0FF0DF
:101ED80053EF0FF081EF0FF065512CEC17F024C091
:101EE80062F025C063F0F29E62C0D9FF63C0DAFFDA
:101EF800000EDE6E000EDD6EF28E95EC1CF0000E0C
:101F080012008FEC1AF00001656F6551D8A48FEFAD
:101F18000FF091EF0FF094EF0FF0020EDAEF0FF0E1
:101F28000F0E65659AEF0FF09CEF0FF09EEF0FF024
:101F380091EF0FF00F0E6519D8A4A5EF0FF0A7EFDA
:101F48000FF0C6EF0FF0010E646F64510BEC17F041
:101F580024C060F025C061F0F29E60C0D9FF61C066
:101F6800DAFF000EDE6E000EDD6EF28E0001642BCD
:101F78000E0E6465C2EF0FF0C4EF0FF0A9EF0FF07B
:101F8800D7EF0FF065510BEC17F024C062F025C0B5
:101F980063F0F29E62C0D9FF63C0DAFF000EDE6E06
:101FA800000EDD6EF28E95EC1CF0000E1200660E2F
:101FB8001D6E000E1E6E0001B251FCEC13F0000104
:101FC80020EE01F06651D9266751DA22DF50616FA1
:101FD800010E6BEC15F098EC1CF0300E46EC1BF083
:101FE8000001615146EC1BF0000E0001656F1BEF0C
:101FF80010F0000E6525D96EDA6A030EDA22DF507A
:10200800646F64390F0B0F0BCBEC18F00001626F93
:1020180064510F0BCBEC18F00001636F625146EC72
:102028001BF00001635146EC1BF00001652B2F509B
:10203800655DD8A022EF10F024EF10F0FDEF0FF04F
:10204800C3EC1CF06BEC15F0000E6BEC15F01200F5
:10205800236E57EF10F0040E1F6E010E206E7CEFFA
:1020680010F0140E1F6E010E206E7CEF10F0240E7F
:102078001F6E010E206E7CEF10F0340E1F6E010EE5
:10208800206E7CEF10F0440E1F6E010E206E7CEF68
:1020980010F0540E1F6E010E206E7CEF10F07FECD6
:1020A80016F02FEF10F02350216E226A2250000AFA
:1020B800D8B461EF10F053EF10F02150090AD8B4EA
:1020C8002FEF10F0030AD8B435EF10F0010AD8B496
:1020D8003BEF10F0070AD8B441EF10F0010AD8B46A
:1020E80047EF10F0030AD8B44DEF10F053EF10F09B
:1020F8001200226E300E1D6E390E1E6E2250E5EC57
:1021080017F00009D8B48BEF10F08DEF10F096EFB0
:1021180010F02250D00F20C0D9FF21C0DAFFDF6EA7
:10212800C9EF10F0610E1D6E660E1E6E2250E5ECB2
:1021380017F00009D8B4A3EF10F0A5EF10F0AEEF38
:1021480010F02250A90F20C0D9FF21C0DAFFDF6E9E
:10215800C9EF10F0410E1D6E460E1E6E2250E5ECC2
:1021680017F00009D8B4BBEF10F0BDEF10F0C6EFC0
:1021780010F02250C90F20C0D9FF21C0DAFFDF6E4E
:10218800C9EF10F0130ECAEF10F0000E1200200E67
:1021980000019827030E9923000E9A23000E9B2313
:1021A8009B510DE1400E985D420E99590F0E9A59B8
:1021B800D8A0E1EF10F0E3EF10F011EF11F0C7EC49
:1021C8001CF00009D8B4EBEF10F0EDEF10F0F1EFD0
:1021D80010F052EC1CF0F3EF10F056EC1CF0010E6E
:1021E8000001A027000EA123A223A323010E9C27F0
:1021F800000E9D239E239F233250D8B406EF11F082
:1022080008EF11F009EF11F03206400E985F420E08
:10221800995B0F0E9A5B000E9B5B1200050EFFEC9C
:1022280017F0000E236E030E216E700E206E5C0EEA
:10223800E82EFED7202EFCD7212EFAD700D0000E8C
:10224800246E24502B0DBF0EF324D96E040EF420F7
:10225800DA6EDECF20F0DDCF21F0050E226ED890A9
:1022680021322032222E33EF11F024502B0DCB0EC9
:10227800F324D96E040EF420DA6E2050DE262150A5
:10228800DD22242A0A0E24644CEF11F04EEF11F0DF
:1022980025EF11F0232A1F0E236455EF11F057EF95
:1022A80011F017EF11F012008FEC1AF0216E020EE8
:1022B800216461EF11F063EF11F071EF11F0020E7C
:1022C8009DEF11F092EC1CF08AEF11F08FEC1CF0EE
:1022D8008AEF11F0010E9DEF11F021501E6E1F6A5A
:1022E8001F50000AD8B47BEF11F06EEF11F01E50AA
:1022F800000AD8B466EF11F0010AD8B46AEF11F0F9
:10230800030AD8B48AEF11F06EEF11F0BFEC1CF09D
:102318000009D8A492EF11F095EF11F0010E96EF95
:1023280011F0000E206E95EC1CF0205084EC1AF091
:10233800000E12001F6EA7EF11F0010EE0EF11F072
:10234800000EE0EF11F01F501D6E1E6A1E50000AAD
:10235800D8B4B1EF11F0A4EF11F01D50010AD8B4B0
:10236800A1EF11F0030AD8B4A1EF11F0010AD8B413
:10237800A1EF11F0070AD8B4A1EF11F0010AD8B4FF
:10238800A1EF11F0030AD8B4A1EF11F0010AD8B4F3
:10239800A1EF11F00F0AD8B4A1EF11F0010AD8B4D7
:1023A800A1EF11F0030AD8B4A1EF11F0010AD8B4D3
:1023B800A1EF11F0A4EF11F012008FEC1AF0276EC4
:1023C8008FEC1AF0266E2750D8A4EDEF11F0EFEF3E
:1023D80011F0F2EF11F0020E20EF12F0020E276456
:1023E800F8EF11F0FAEF11F0FCEF11F0EFEF11F048
:1023F800010E266402EF12F004EF12F006EF12F05D
:10240800EFEF11F0275096EC15F01FC024F020C014
:1024180025F0F29E02D81CEF12F00500FA6E245047
:10242800FD6E2550FE6EF850FF6EFA5026501200D1
:10243800F28E95EC1CF0000E1200000E0001646F85
:10244800000E656F000E666F800E676F000E696F75
:10245800800E686F800E6B6F000E6A6F040E6C6FD3
:10246800400E6D6F95EC1CF0800E1D6E000E1E6EFA
:10247800000E1F6E000E206EC7EC16F0000E1D6ECB
:10248800000E1E6E000E1F6E800E206EC7EC16F03A
:10249800000E1E6E800E1D6E04EC19F0800E1E6E6E
:1024A800000E1D6E04EC19F0040E84EC1AF0400EB8
:1024B80084EC1AF0000E12008D0E1D6E000E1E6EBA
:1024C8000001B251FCEC13F000018C6F8C51D8B4B0
:1024D80070EF12F072EF12F075EF12F0180E9CEF19
:1024E80012F020EE02F08D51D9268E51DA222F50AB
:1024F800DE18D8B482EF12F084EF12F086EF12F0F3
:1025080072EF12F071EC1CF0000120EE03F08D5117
:10251800D9268E51DA2202D89CEF12F00500FA6E05
:10252800DE50FD6EDE50FE6EF850FF6EFA5012005F
:102538001200000E0001656F220E646F070E676FB0
:10254800E70E666F0A0E686F1A0E696F130E6A6FD0
:102558000B0E6B6F000E6C6F95EC1CF0010E1D6E70
:10256800000E1E6E000E1F6E000E206EC7EC16F0D9
:10257800000E1E6E220E1D6E04EC19F0070E1E6E64
:10258800E70E1D6E04EC19F00A0E84EC1AF01A0E10
:1025980084EC1AF0130E84EC1AF00B0E84EC1AF08B
:1025A800000E84EC1AF0000E12008FEC1AF00001F5
:1025B800656F6551D8A4E3EF12F0E5EF12F0E8EF8C
:1025C80012F0020E13EF13F0080E6565EEEF12F02D
:1025D800F0EF12F0F2EF12F0E5EF12F065C064F0E0
:1025E8006551AEEC0AF01FC060F020C061F0000138
:1025F80020EE02F06051D9266151DA22DECF62F076
:10260800DDCF63F095EC1CF00001645184EC1AF006
:1026180062C01DF063C01EF004EC19F0000E120039
:102628008FEC1AF00001656F6551D8A41EEF13F006
:1026380020EF13F023EF13F0020E4DEF13F00E0E00
:10264800656529EF13F02BEF13F02DEF13F020EF52
:1026580013F065C064F065512CEC17F024C062F0EB
:1026680025C063F0F29E62C0D9FF63C0DAFFDECFF7
:1026780060F0DDCF61F0F28E95EC1CF00001645142
:1026880084EC1AF060C01DF061C01EF004EC19F073
:10269800000E12008FEC1AF00001656F6551D8A486
:1026A80058EF13F05AEF13F05DEF13F0020E87EFB7
:1026B80013F00E0E656563EF13F065EF13F067EF27
:1026C80013F05AEF13F065C064F065510BEC17F086
:1026D80024C062F025C063F0F29E62C0D9FF63C0D7
:1026E800DAFFDECF60F0DDCF61F0F28E95EC1CF002
:1026F8000001645184EC1AF060C01DF061C01EF046
:1027080004EC19F0000E12008FEC1AF00001656F4E
:102718006551D8A492EF13F094EF13F097EF13F0EC
:10272800020EC1EF13F00E0E65659DEF13F09FEFDB
:1027380013F0A1EF13F094EF13F065C064F0655146
:10274800EAEC16F024C062F025C063F0F29E62C085
:10275800D9FF63C0DAFFDECF60F0DDCF61F0F28E23
:1027680095EC1CF00001645184EC1AF060C01DF077
:1027780061C01EF004EC19F0000E12009D9A8E0E36
:102788001D6E180E1E6EC8EC1BF09D981E0E1D6E59
:102798002F0E1E6EC3EC1BF0080EB86E900EAB6EBB
:1027A800240EAC6E400EAF6E030EB06E9E0E1D6E04
:1027B800390E1E6ED2EC1BF0660E1D6E390E1E6EA3
:1027C800CDEC1BF06C0E1D6E390E1E6ED7EC1BF097
:1027D800000E366E000E3C6E000E3B6E400E3A6EDA
:1027E800000E396E000E386E000E376E9D8A12008C
:1027F800226EC1EC1CF0236E1DC0D9FF1EC0DAFF8B
:10280800000EDE6E040EDD6E2AEF14F01DC0D9FF37
:102818001EC0DAFFDECF1FF0DDCF20F01FC0D9FFCA
:1028280020C0DAFF2250DE18D8A41DEF14F01FEFE5
:1028380014F022EF14F0000E34EF14F0050E1DC052
:10284800D9FF1EC0DAFFDE26000EDD22230623286C
:10285800D8A431EF14F033EF14F00AEF14F0200E7F
:1028680012008FEC1AF00001646FAFEC17F01DC076
:1028780060F01EC061F000016451D8A446EF14F066
:1028880048EF14F04BEF14F0020E6CEF14F0080E42
:10289800646551EF14F053EF14F055EF14F048EF5E
:1028A80014F06451AEEC0AF01FC062F020C063F06F
:1028B800F29E000120EE02F06251D9266351DA221D
:1028C80060C0DEFF61C0DDFFF28E95EC1CF0000EEB
:1028D80012001F6E76EF14F0010EA3EF14F0000E35
:1028E800A3EF14F01F501D6E1E6A1E50000AD8B4C4
:1028F80080EF14F073EF14F01D50010AD8B470EF94
:1029080014F0030AD8B470EF14F0010AD8B470EFC9
:1029180014F0070AD8B470EF14F0010AD8B470EFB5
:1029280014F0030AD8B470EF14F0010AD8B470EFA9
:1029380014F00F0AD8B470EF14F073EF14F012000B
:102948008FEC1AF00001656FAFEC17F01DC061F055
:102958001EC062F000016551D8A4B5EF14F0B7EFBE
:1029680014F0BAEF14F0020ED8EF14F00E0E6565ED
:10297800C0EF14F0C2EF14F0C4EF14F0B7EF14F086
:102988006551EAEC16F024C063F025C064F0F29EAD
:1029980063C0D9FF64C0DAFF61C0DEFF62C0DDFF3B
:1029A800F28E95EC1CF0000E1200000E0001806FF4
:1029B8008FEC1AF01E6E600E00018025D96EDA6A5F
:1029C800000EDA221EC0DFFF802B1F0E8065EFEF9E
:1029D80014F0F1EF14F0DCEF14F095EC1CF0000E9D
:1029E8000001806F600E8025D96EDA6A000EDA2247
:1029F800DF5084EC1AF00001802B1F0E806507EF72
:102A080015F009EF15F0F6EF14F0000E12009AEC2D
:102A18001AF00009D8B413EF15F015EF15F019EFF7
:102A280015F00FEC16F090EC00F061EC1AF00009CC
:102A3800D8B421EF15F023EF15F03AEF15F060EC5C
:102A480012F000018F6F8F51D8A42DEF15F02FEFE2
:102A580015F035EF15F049EC1AF0DBEC0FF038EF14
:102A680015F08F5136EC1CF0B0EC1AF0120095EC12
:102A78001CF0010E0001656F000E646F65512CECAF
:102A880017F024C062F025C063F0F29E62C0D9FF3F
:102A980063C0DAFFDE50DE10D8B455EF15F057EFFB
:102AA80015F05AEF15F0010E0001646FF28E000167
:102AB800645184EC1AF00001652B0E0E656567EF12
:102AC80015F069EF15F040EF15F0000E12001D6EBD
:102AD8003A50D8B472EF15F074EF15F06CEF15F0AA
:102AE8009DB879EF15F07BEF15F07FEF15F01DC05D
:102AF800ADFF94EF15F09D98400E3C24D96EDA6A2C
:102B0800020EDA221DC0DFFF3C2A3F0E3C648FEF25
:102B180015F091EF15F093EF15F0000E3C6E3A06A4
:102B28009D881200236EA5EF15F01E0E1F6E330E42
:102B3800206EBEEF15F0FE0E1F6E320E206EBEEF39
:102B480015F02350216E226A2250000AD8B4AFEF44
:102B580015F0BAEF15F02150010AD8B499EF15F025
:102B6800030AD8B49FEF15F0BAEF15F07FEC16F012
:102B78009FEF15F0120095EC1CF0010E0001646F38
:102B880064510BEC17F024C060F025C061F0F29E90
:102B980060C0D9FF61C0DAFFDECF62F0DDCF63F03D
:102BA800F28E62C01DF063C01EF004EC19F0000143
:102BB800642B0E0E6465E3EF15F0E5EF15F0C4EF36
:102BC80015F0000E120095EC1CF0010E0001646F68
:102BD80064512CEC17F024C060F025C061F0F29E1F
:102BE80060C0D9FF61C0DAFFDECF62F0DDCF63F0ED
:102BF800F28E62C01DF063C01EF004EC19F00001F3
:102C0800642B0E0E64650BEF16F00DEF16F0ECEF6B
:102C180015F0000E12003750D8B415EF16F017EF64
:102C280016F00FEF16F0C00E3824D96EDA6A010ECE
:102C3800DA22DF50366E000E3824D96EDA6A020EB8
:102C4800DA22DF501D6E382A3F0E38642EEF16F058
:102C580030EF16F032EF16F0000E386E9D9A3706F8
:102C68009D8A1D50120095EC1CF0010E0001636F47
:102C780063514DEC17F024C060F025C061F0F29E5E
:102C880060C0D9FF61C0DAFFDF500001626FF28EC9
:102C9800625184EC1AF00001632B0E0E636557EF46
:102CA80016F059EF16F03CEF16F0000E12008FECFC
:102CB8001AF01E6E8FEC1AF01F6E8FEC1AF0206E51
:102CC8008FEC1AF0216E1EC022F01FC023F020C026
:102CD80024F021C025F095EC1CF0225084EC1AF069
:102CE800235084EC1AF0245084EC1AF0255084EC1C
:102CF8001AF0000E1200F29E3EEC1CF046EC1CF09E
:102D0800150E1E6E4B0E1D6EBE0EE82EFED71D2E26
:102D1800FCD71E2EFAD700D03AEC1CF042EC1CF07F
:102D2800150E1E6E4B0E1D6EBE0EE82EFED71D2E06
:102D3800FCD71E2EFAD700D080EF16F01200F29EB4
:102D480056EC1CF05AEC1CF0150E026E4B0E016E80
:102D5800BE0EE82EFED7012EFCD7022EFAD700D0E1
:102D680052EC1CF05EEC1CF0150E026E4B0E016E60
:102D7800BE0EE82EFED7012EFCD7022EFAD700D0C1
:102D8800A4EF16F01200000E2F24D96EDA6A030E93
:102D9800DA2220C0DFFF010E2F24D96EDA6A030E73
:102DA800DA221FC0DFFF020E2F24D96EDA6A030E63
:102DB800DA221EC0DFFF030E2F24D96EDA6A030E53
:102DC800DA221DC0DFFF040E2F261200266E2650C1
:102DD8006DEC14F00009D8B4F4EF16F0F6EF16F025
:102DE80001EF17F02650AEEC0AF0040E1F24246EF3
:102DF800000E2020256E0AEF17F026502CEC10F05C
:102E0800020E1F24246E000E2020256E1200266E4E
:102E180026506DEC14F00009D8B415EF17F017EF31
:102E280017F022EF17F02650AEEC0AF0080E1F2418
:102E3800246E000E2020256E2BEF17F026502CEC68
:102E480010F0060E1F24246E000E2020256E12009E
:102E5800266E26506DEC14F00009D8B436EF17F042
:102E680038EF17F043EF17F02650AEEC0AF00A0ED1
:102E78001F24246E000E2020256E4CEF17F02650DC
:102E88002CEC10F00A0E1F24246E000E2020256E54
:102E98001200266E26506DEC14F00009D8B457EFD6
:102EA80017F059EF17F064EF17F02650AEEC0AF060
:102EB800010E1F24246E000E2020256E6DEF17F0E2
:102EC80026502CEC10F0010E1F24246E000E20203A
:102ED800256E1200000E8D6E000E8C6E000E896E2F
:102EE800000E8A6E000E8B6E070E966E3F0E926E67
:102EF8009368BF0E946E000E956E0F013B69000E2D
:102F08003A6F0E0E396F070E3C6F2F0E386F000E9A
:102F1800616EF18E1200400E3A6095EF17F097EF50
:102F280017F0ADEF17F0400E3B24D96EDA6A020EA7
:102F3800DA22DF50AD6E3B2A3F0E3B64A6EF17F056
:102F4800A8EF17F0AAEF17F0000E3B6E3A2AAEEF83
:102F580017F09D981200010E2F24D96EDA6A030E1D
:102F6800DA22DF501F6E000E2F24D96EDA6A030EA4
:102F7800DA22DF50206E1F50226E20C023F0020E8E
:102F88002F2622C01DF023C01EF01200F2943DC06F
:102F9800D6FF0001AE51AF11D8B4D5EF17F0D7EF77
:102FA80017F0E4EF17F002D8E4EF17F00500FA6E17
:102FB800AE51FD6EAF51FE6EF850FF6EFA50120022
:102FC80012001F6E1F501E5CD8B0EDEF17F0EFEF28
:102FD80017F0F2EF17F0000EFEEF17F01D501F5C10
:102FE800D8B0F9EF17F0FBEF17F0FDEF17F0EFEFA0
:102FF80017F0010E12001F6E0EEF18F0250E1E6E50
:10300800490E1D6E350EE82EFED71D2EFCD71E2E3E
:10301800FAD700F01F061F28D8A415EF18F017EFED
:1030280018F002EF18F01200DEEC18F01DC060F086
:103038001EC061F01FC062F020C063F095EC1CF068
:1030480060C01DF061C01EF062C01FF063C020F0B8
:10305800C7EC16F0000E1200F1EC18F01DC060F07D
:103068001EC061F01FC062F020C063F095EC1CF038
:1030780060C01DF061C01EF062C01FF063C020F088
:10308800C7EC16F0000E12009E9228502910D8B4F2
:1030980050EF18F052EF18F05FEF18F002D85FEF1A
:1030A80018F00500FA6E2850FD6E2950FE6EF85093
:1030B800FF6EFA501200120076EC18F09BEC1CF030
:1030C800DCEC1BF03DEC19F012EC11F0CCEC1CF030
:1030D8002AEC19F0D8EC0EF00BEC15F06EEF18F0A6
:1030E8008EEF00F017EC19F03A0E1D6E380E1E6EBA
:1030F800BEEC1BF0420E1D6E390E1E6EB9EC1BF0B5
:10310800D00E1F6ECA0EE82EFED71F2EFCD7120057
:10311800000E096E0950100D000EF324036E010E07
:10312800F420046EB8EC01F0092A0B0E09649FEF35
:1031380018F0A1EF18F08EEF18F01200000E3924E5
:10314800D96EDA6A020EDA22AECFDFFF392A3F0ED5
:103158003964B1EF18F0B3EF18F0B5EF18F0000EBE
:10316800396E372A1200BDEC1CF00009D8A4BFEF55
:1031780018F0C2EF18F0010EC3EF18F0000E1E6E23
:1031880095EC1CF01E5084EC1AF0000E12001D6E17
:103198001D500F0B1D6E0A0E1D60D5EF18F0D7EFEE
:1031A80018F0DBEF18F01D50300FDDEF18F01D5050
:1031B800570F1200F29EA0C021F0A1C022F0A2C0B9
:1031C80023F0A3C024F0F28E21C01DF022C01EF00F
:1031D80023C01FF024C020F01200F29E9CC021F0F2
:1031E8009DC022F09EC023F09FC024F0F28E21C023
:1031F8001DF022C01EF023C01FF024C020F01200D2
:10320800000E2F24D96EDA6A030EDA221E50DF6E02
:10321800010E2F24D96EDA6A030EDA221DC0DFFFF1
:10322800020E2F261200C5EC1CF06EEC17F02EECE7
:103238001AF04EEC1CF0A5EC1AF04EEC1BF01FEC4B
:103248001AF04EEC19F0C2EC13F01200050EFFEC68
:1032580017F0010EBFEC19F0780EFFEC17F0010E15
:10326800AFEC19F0780EFFEC17F0010E9FEC19F097
:103278001200F28EF28C9AEC1AF00009D8A447EFEB
:1032880019F049EF19F03FEF19F0BBEC1CF0B9EC5D
:103298001CF01200000ED76E380ED66E380E3D6E3A
:1032A800F294F28A9C0E1D6E390E1E6EBEEC1BF057
:1032B800D50ED56E1200AFEC17F01DC024F01EC05D
:1032C80025F024C01DF025C01EF0AFEC1BF095ECD6
:1032D8001CF0000E1200B4EC1BF01DC01FF01EC045
:1032E80020F095EC1CF01FC01DF020C01EF004EC6F
:1032F80019F0000E12001D6E1D04D8A486EF19F0F7
:1033080088EF19F08CEF19F046EC1CF08EEF19F0ED
:1033180042EC1CF012001D6E1D04D8A496EF19F0A3
:1033280098EF19F09CEF19F03EEC1CF09EEF19F0A5
:103338003AEC1CF012001D6E1D04D8A4A6EF19F07B
:10334800A8EF19F0ACEF19F0E6EC1BF0AEEF19F0AE
:10335800E1EC1BF012001D6E1D04D8A4B6EF19F0A5
:10336800B8EF19F0BCEF19F0F0EC1BF0BEEF19F054
:10337800EBEC1BF012001D6E1D04D8A4C6EF19F06B
:10338800C8EF19F0CCEF19F0FAEC1BF0CEEF19F0FA
:10339800F5EC1BF012001D6E1D04D8A4D6EF19F031
:1033A800D8EF19F0DCEF19F0A0EC1BF0DEEF19F004
:1033B8009BEC1BF012001D6E1D04D8A4E6EF19F05B
:1033C800E8EF19F0ECEF19F096EC1BF0EEEF19F0BE
:1033D80091EC1BF012001D6E1D04D8A4F6EF19F035
:1033E800F8EF19F0FCEF19F0AAEC1BF0FEEF19F05A
:1033F800A5EC1BF012001D6E1D04D8A406EF1AF0F0
:1034080008EF1AF00CEF1AF08CEC1BF00EEF1AF024
:1034180087EC1BF012001D6E1D04D8A416EF1AF0DD
:1034280018EF1AF01CEF1AF082EC1BF01EEF1AF0DE
:103438007DEC1BF01200C70EBB6E000EBC6E9E9298
:103448009D829A0E1D6E390E1E6EB9EC1BF01D0E74
:10345800BA6E1200700ED36E040ED26E400E9B6EC2
:10346800D2AE39EF1AF03BEF1AF034EF1AF012002F
:10347800F29E3EC01EF0000E3E6EF28E95EC1CF0E1
:103488001E5084EC1AF0000E1200F29E000E00018D
:10349800A06F000EA16F000EA26F000EA36FF28E38
:1034A80012008FEC1AF01E6E1EC01FF095EC1CF077
:1034B8001F5084EC1AF0000E1200070E3118D8B411
:1034C80068EF1AF06BEF1AF0010E6CEF1AF0000EAD
:1034D8001200026E02C001F001460146C2500118F6
:1034E800830B0118C26EC2801200F29E42C01EF009
:1034F800F28E95EC1CF01E5084EC1AF0000E1200AF
:103508001D6E000E2F24D96EDA6A030EDA221DC052
:10351800DFFF2F2A1200000E2F24D96EDA6A030E5D
:10352800DA22DF501D6E2F2A1D5012003750D8A402
:10353800A0EF1AF0A3EF1AF0010EA4EF1AF0000E94
:103548001200080EC16E3D0EC06E000EC36E000E56
:10355800C46E010EC26E1200000E316EFE0E000126
:10356800B26F000E306E000E2F6E120081B0BFEFEA
:103578001AF0C2EF1AF0010EC3EF1AF0000E120093
:1035880082BAC9EF1AF0CCEF1AF0010ECDEF1AF09B
:10359800000E120082A8D3EF1AF0D6EF1AF0010E2F
:1035A800D7EF1AF0000E120082A6DDEF1AF0E0EF56
:1035B8001AF0010EE1EF1AF0000E120082A4E7EFF4
:1035C8001AF0EAEF1AF0010EEBEF1AF0000E1200F3
:1035D80082A2F1EF1AF0F4EF1AF0010EF5EF1AF0EB
:1035E800000E120080A8FBEF1AF0FEEF1AF0010E91
:1035F800FFEF1AF0000E120081BE05EF1BF008EF76
:103608001BF0010E09EF1BF0000E120081BC0FEF3A
:103618001BF012EF1BF0010E13EF1BF0000E12004F
:1036280081BA19EF1BF01CEF1BF0010E1DEF1BF008
:10363800000E120081B823EF1BF026EF1BF0010EDD
:1036480027EF1BF0000E120082B02DEF1BF030EFB9
:103658001BF0010E31EF1BF0000E1200C2A237EF73
:103668001BF03AEF1BF0010E3BEF1BF0000E1200AF
:10367800C450046E036AC3500324016E000E042074
:10368800026E12001E6E1E506BEC15F01E504AECB6
:103698001CF01200000E0F01546F000E556F000E43
:1036A800566F1200D638D038CA38C438DC38DC0532
:1036B8000004226E225036EC1CF0B0EC1AF0120016
:1036C800000E356E000E346E410E336E12001D6E04
:1036D800F29E1DC032F0F28E1200F29E32C01DF032
:1036E800F28E1D5012008CEC1CF095EC1CF0000EB4
:1036F80012008C90000E0001906F12008C80010E59
:103708000001906F12008C92000E0001916F120060
:103718008C82010E0001916F12008C96000E000140
:10372800936F12008C86010E0001936F12008C9823
:10373800000E0001946F12008C88010E0001946F36
:1037480012008C94000E0001926F12008C84010EFE
:103758000001926F12001DC0BDF01EC0BEF0120025
:10376800BDC01DF0BEC01EF012001DC028F01EC056
:1037780029F012001DC0AEF01EC0AFF012001DC02F
:10378800AAF01EC0ABF012001DC0ACF01EC0ADF018
:1037980012001DC0A6F01EC0A7F012001DC0A8F0A0
:1037A8001EC0A9F012001DC0A4F01EC0A5F0120092
:1037B80064EC1BF09EEC1CF012008C9E000E0001C5
:1037C800976F12008C8E010E0001976F12008C9C6F
:1037D800000E0001966F12008C8C010E0001966F8E
:1037E80012008C9A000E0001956F12008C8A010E4F
:1037F8000001956F120022EC1CF027EC1CF012005F
:1038080022EC1CF027EC1CF0120022EC1CF027EC38
:103818001CF0120022EC1CF027EC1CF0120022EC29
:103828001CF027EC1CF0120022EC1CF027EC1CF01A
:10383800120088EC08F0CBEC10F012008C90000E0F
:103848000001906F12008C92000E0001916F12001F
:103858008C96000E0001936F12008C98000E0001E8
:10386800946F12001D6E1DC03EF01200899E000E5E
:103878002A6E1200898E010E2A6E1200899C000E93
:103888002B6E1200898C010E2B6E12001D6E1D50BE
:103898002E5E1200B00E0F01426F1200899E000EBC
:1038A8002A6E1200898E010E2A6E1200899C000E63
:1038B8002B6E1200898C010E2B6E1200A0EC1BF0EF
:1038C8001200AAEC1BF0120082EC1BF012008CEC28
:1038D8001BF0120096EC1BF01200000E2F6E120067
:1038E80000019751120000019651120000019551F4
:1038F80012000001945112000001935112000001BE
:1039080092511200000191511200000190511200D1
:10391800000E2D6E1200010E416E1200000E416E57
:103928001200000E2F6E1200000E2E6E1200B0EC68
:103938001AF01200010E356E12008CEC18F012000D
:103948002CEC1CF0120031EC1CF0120031EC1CF0D5
:103958001200A3EC16F012002CEC1CF01200AB982D
:10396800AB881200A2EC18F01200BA841200D58EAF
:1039780012002D50120041501200260E12002E5037
:103988001200D09E12002A501200C2821200010AB0
:083998001200120012001200DF
:020000040020DA
:08000000FFFFFFFFFFFFFFFF00
:020000040030CA
:0E000000FF281F3CFFBF85FF0FC00FE00F4021
:00000001FF
